:0E00000022C0FECF5BC0FCCFFBCF3AC0F9CFD1
:10000E00F8CFF7CFF6CFF5CFF4CFF3CFF2CFF1CFC6
:10001E00F0CFEFCFEECFEDCFECCFEBCF1027E80345
:10002E0064000A0001000010000110000100726659
:10003E00496E69740D0A0000F894EE27ECBBE5BF1B
:10004E00F8E1A895A4B7A77FA4BFF1BDE1BD8DE0EF
:10005E00A2E0ED938A95E9F780E8A0E6ED938A9504
:10006E00E9F7E0E0E3BBE4BBE5BBEFEDEDBFC0E8D5
:10007E005BC1AA93EA93EFB7EA93EFE1EDBDE0E03F
:10008E00ECBDA0E09899A1E0E1E0EA2711F4989880
:10009E0001C0989A849B06C03394E2E0E31511F4F4
:1000AE0094983324E991EFBFE991A99118950A929A
:1000BE001A92FA926A937A938A939A93AA93BA931C
:1000CE00EA93FA93EFB7EA93E0E0EBBF839902C0AD
:1000DE00859901C002C0A1E057D1839902C0859BCA
:1000EE0001C002C0A2E050D1E0E8EBBFE991EFBF42
:1000FE00F991E991B991A991999189917991699122
:10010E00F990199009901895BA93AA931A9310E042
:10011E00EB811E1750F4969AA981BA8191D19698C7
:10012E00A981BA818DD11F5FF3CF188156C0BA93C2
:10013E00AA9390D100E010E0C498EB81F070EFB973
:10014E00E1E1EDB9E3E1EDB9E1E1EDB9E3E1EDB9FD
:10015E00E1E1EDB9E3E1EDB9E1E1EDB9E3E1EDB9ED
:10016E00E1E1EDB9E3E1EDB9E1E1EDB9E3E1EDB9DD
:10017E00E1E1EDB9E3E1EDB9E1E1EDB9E3E1EDB9CD
:10018E00EFB1FE2FE0E08F01EA81EFB9E1E1EDB9C9
:10019E00E3E1EDB9E1E1EDB9E3E1EDB9E1E1EDB9AD
:1001AE00E3E1EDB9E1E1EDB9E3E1EDB9E1E1EDB99D
:1001BE00E3E1EDB9E1E1EDB9E3E1EDB9E1E1EDB98D
:1001CE00E3E1EDB9E1E1EDB9E3E1EDB9EFB1F0E075
:1001DE000E2B1F2BC49AF80140D124960895AA9392
:1001EE008299FECFE881EFB9E1E1EDB9E3E1EDB936
:1001FE00E1E1EDB9E3E1EDB9E1E1EDB9E3E1EDB94D
:10020E00E1E1EDB9E3E1EDB9E1E1EDB9E3E1EDB93C
:10021E00E1E1EDB9E3E1EDB9E1E1EDB9E3E1EDB92C
:10022E00E1E1EDB9E3E1EDB9F4C0A0E0BEEF7FDFAF
:10023E00A6E9B0E005D1A8EDB0E879DFA9EDB2E806
:10024E0076DFA0E2B6EA73DFA5E0B6EC70DFA0EAD7
:10025E00B4E96DDFACEEB2EC6ADFA3E8BAEC67DFAF
:10026E00A6EDBEEC64DFABE9B4EC61DFA0E5B8E966
:10027E005EDFA7E7BCEC5BDFA0E0B0EE58DFA0E0EE
:10028E00B8EC55DFA0E0B0EC15C0C698B39B02C029
:10029E00B19901C0FBCFC298C498E0E4EEB9EBE18E
:1002AE00EDB9769BFCCFEFB10895A1E8BAEC3FDF34
:1002BE00A3E8BAEC3CDF0895E0E8E6BDE0E0E6BD79
:1002CE00E4E0EBBBE0E0EABBE4E1E8BBE4EDE7BB76
:1002DE00E2E5E1BBEDE2E2BBE0E0E0BFE3BFE2BF9F
:1002EE00E6BFECBFEFBDE4E0EEBDEFE1EDBDE0E05B
:1002FE00ECBDE5BDE4BDEBBDEABDE9BDE8BDE0E8A2
:10030E00E9BFE0E0E5BFE0E8EBBFEABFE0E0EDB952
:10031E00EBB9E8E1EAB9E6E0E3B9E0E0E2B9E0E83A
:10032E00E8B9E0E0E1B90895F894C6DFE7E0E9B98D
:10033E007CDFACE3B0E06FD0E3E0EA93A4E6B0E09C
:10034E00E3DE7894B2DFA1DF1E2FA12F5DD01B3626
:10035E00B1F49BDF0E2F99DF3E2F97DF2E2F95DF07
:10036E005E2FC29AC49AA1DF013331F4323321F4E5
:10037E00233311F4543309F001C0949AE4CFC29A96
:10038E00C49A93DFE0CFFFCFFF92AA93869907C05E
:10039E006894F0F8969AC29AA9E3B2E8C8DEC29AB7
:1003AE00A0E0B0E0C4DEC498A8EB19DFAAEA17DF1C
:1003BE00ADE215DFA6ED13DFABE611DFA881A130AC
:1003CE0041F4A1E30CDFA2E30ADFA3E308DFA4E319
:1003DE0006DFA881A23041F4A2E301DFA5E3FFDE30
:1003EE00A7E3FDDEA2E3FBDEA0E0F9DEC298C49A2D
:1003FE00A9E1B0E025D0F0FE04C0A9EDB2E897DE89
:10040E0096982196FF900895AA935D9BFECFE88162
:10041E00ECB921960895BA93AA931A93E981FA81B9
:10042E003196E983FA833197E4911E2FE03019F06B
:10043E00A12FEADFF3CFAAE0E7DF18812396089514
:10044E00109639F086E69EE00197F1F7A895119780
:10045E00C9F708951A930A9308951981088108958A
:00000001FF
